:020000040000FA
:0400000001303A2869
:08000800A000030EA100831209
:1000100081018B100B11210E8300A00E200E090010
:0C007400203084008001840A6030040207
:10008000031C3C281230B00058218316FF23900037
:10009000831283160C308505870183128501870141
:1000A000073099000030831691009F008312C830FA
:1000B00083168100831231309000003083168C004B
:1000C000831210308B00831610309B001C141A080A
:1000D0008312BD00BE2181018E018F010B118B1097
:1000E0000B108C018B178720311989203C21B30B11
:1000F0008528031085190314B90DF030390203194E
:10010000D5210F3039020319CF21DF217328640074
:100110000800080031110130B7008B132030370779
:1001200083169B001C141A088312A4001030370792
:1001300083169B001C141A088312A3000030370793
:1001400083169B001C141A088312A2008B17321C02
:10015000AF2822090339A200A309A409A509013087
:100160003702031DB6283D143E14602102303702C9
:10017000031DBD28BD143E146C2103303702031D3E
:10018000C4283D153E14782104303702031DCB28C6
:10019000BD153E14842101303702031DD2283D10C5
:1001A0003E14902102303702031DD928BD103E14A1
:1001B000992103303702031DE0283D113E14A2218E
:1001C00004303702031DE728BD113E14AB21E82897
:1001D000B70A05303702031808008D280130B60031
:1001E000B300B400B500B70085018701B1138720C3
:1001F000B30B1429031085190314B90DF03039021B
:1002000003193229B41F8501B41F8701B40B1429C7
:100210003708B6080319B60003191229FF30850004
:100220008700B6039630B400311DF7283111321C17
:100230001E292D090339AD00AE09AF098B132030FB
:100240003707BB002F08BA00452110303707BB0025
:100250002E08BA00452100303707BB002D08BA0030
:1002600045218B1785018701B70AB6010530370292
:10027000031CF728BE2108003E1C08003E10103069
:10028000BB003D08BA00452108008B133A088316CD
:100290001C159A003B089B0055309D00AA309D001C
:1002A0009C1464009C1851291C1183128B170800A0
:1002B000831610309B001C141A088312BD0008001E
:1002C0003D14A222DC00B222C400C222CC000130C4
:1002D000C800FF30C0000800BD14A622DD00B62211
:1002E000C500C622CD000130C900FF30C1000800A2
:1002F0003D15AA22DE00BA22C600CA22CE00013075
:10030000CA00FF30C2000800BD15AE22DF00BE22C9
:10031000C700CE22CF000130CB00FF30C300080061
:100320005C1A8510DC1A05105C1B8512DC1B05129B
:1003300008005D1A8510DD1A05105D1B8512DD1B96
:10034000051208005E1A8510DE1A05105E1B851264
:10035000DE1B051208005F1A8510DF1A05105F1BEF
:100360008512DF1B05120800380903398500B80023
:100370000800380930398500B80008003D186021B0
:100380005C1C3D10BD186C215D1CBD103D19782111
:100390005E1C3D11BD1984215F1CBD1108003D1874
:1003A00008003D1460213E1408003D109021BD104E
:1003B00099213D11A221BD11AB213E1408000A3044
:1003C0000F02031C08008E018F013D1C0F2AC80B71
:1003D0000F2A4C08C800C00A4408400203180B2A20
:1003E0008E22D0005C1EF829501C851050188514F0
:1003F000DC1EFE29D01C0510D01805145C1F042A31
:10040000501D851250198516DC1F0F2AD01D0512AC
:10041000D01905160F2AC0015C18F0293D10BD1C2B
:10042000392AC90B392A4D08C900C10A45084102B9
:100430000318352A9322D0005D1E222A501C8510F5
:1004400050188514DD1E282AD01C0510D01805145C
:100450005D1F2E2A501D851250198516DD1F392A61
:10046000D01D0512D0190516392AC1015D181A2AA6
:10047000BD103D1D632ACA0B632A4E08CA00C20A7A
:100480004608420203185F2A9822D0005E1E4C2ABA
:10049000501C851050188514DE1E522AD01C0510E1
:1004A000D01805145E1F582A501D85125019851644
:1004B000DE1F632AD01D0512D0190516632AC2015A
:1004C0005E18442A3D11BD1D8D2ACB0B8D2A4F0885
:1004D000CB00C30A470843020318892A9D22D00093
:1004E0005F1E762A501C851050188514DF1E7C2A4A
:1004F000D01C0510D01805145F1F822A501D8512CC
:1005000050198516DF1F8D2AD01D0512D01905162A
:100510008D2AC3015F186E2ABD11080003308A00BE
:100520004008003E820003308A004108403E8200BD
:1005300003308A004208803E820003308A0043086C
:10054000C03E820003308A003730820003308A00C8
:100550007730820003308A00B730820003308A008F
:10056000F730820003308A003530820003308A0081
:100570007530820003308A00B530820003308A0073
:10058000F530820003308A003630820003308A0062
:100590007630820003308A00B630820003308A0051
:0405A000F6308200AF
:100600000134023403340434053406340734083426
:1006100009340A340B340C340D340E340F341034D6
:100620001134123413341434153416341734183486
:1006300019341A341B341C341D341E341F34203436
:1006400021342234233424342534263427342834E6
:1006500029342A342B342C342D342E342F34303496
:100660003134323441344234433432342834F13476
:100670008034803480348034803480348034FF345B
:1006800001340234033404340534063407340834A6
:1006900009340A340B340C340D340E340F34103456
:1006A0001134123413341434153416341734183406
:1006B00019341A341B341C341D341E341F342034B6
:1006C0002134223423342434253426342734283466
:1006D00029342A342B342C342D342E342F34303416
:1006E0003134323480348034803432341E34303407
:1006F0008034803480348034803480348034FF34DB
:100700000134023403340434053406340734083425
:1007100009340A340B340C340D340E340F341034D5
:100720001134123413341434153416341734183485
:1007300019341A341B341C341D341E341F34203435
:1007400021342234233424342534263427342834E5
:1007500029342A342B342C342D342E342F34303495
:100760003134323480348034803432340A34F134D9
:100770008034803480348034803480348034FF345A
:1007800001340234033404340534063407340834A5
:1007900009340A340B340C340D340E340F34103455
:1007A0001134123413341434153416341734183405
:1007B00019341A341B341C341D341E341F342034B5
:1007C0002134223423342434253426342734283465
:1007D00029342A342B342C342D342E342F34303415
:1007E0003134323480348034803432341434F1344F
:0E07F00080348034803480348034803480340F
:084000000F000300050003009E
:02400E00CC01E3
:10420000FF00FF00FF00FF00FF00FF00FF00FF00B6
:10421000FF00FF00FF00FF00FF00FF00FF00FF00A6
:104220000100FF00FF00FF00FF00FF00FF00FF0094
:10423000FF00FF00FF00FF00FF00FF00FF00FF0086
:104240001000FF00FF00FF00FF00FF00FF00FF0065
:10425000FF00FF00FF00FF00FF00FF00FF00050060
:10426000FF00FF00FF00FF00FF00FF00FF00FF0056
:10427000FF00FF00FF00FF00FF00FF00FF00FF0046
:10428000FF00FF00FF00FF00FF00FF00FF00FF0036
:10429000FF00FF00FF00FF00FF00FF00FF00FF0026
:1042A000FF00FF00FF00FF00FF00FF00FF00FF0016
:1042B000FF00FF00FF00FF00FF00FF00FF00FF0006
:1042C000FF00FF00FF00FF00FF00FF00FF00FF00F6
:1042D000FF00FF00FF00FF00FF00FF00FF00FF00E6
:1042E000FF00FF00FF00FF00FF00FF00FF00FF00D6
:1042F000FF00FF00FF00FF00FF00FF00FF000000C5
:00000001FF
